:020000040800F2
:1000000000060020E1010008E3010008E301000808
:10001000E3010008E3010008E3010008E301000830
:10002000E3010008E3010008E30100085536000879
:10003000E3010008E3010008E3010008E301000810
:10004000E3010008E3010008E3010008E301000800
:10005000E3010008E3010008E3010008E3010008F0
:10006000E3010008E3010008E3010008E3010008E0
:10007000E3010008E3010008E3010008E3010008D0
:10008000E3010008E3010008E3010008E3010008C0
:10009000E3010008E3010008E3010008E3010008B0
:1000A000E3010008E3010008E3010008E3010008A0
:1000B000E3010008E3010008E3010008E301000890
:1000C000E3010008E3010008E3010008E301000880
:1000D000E3010008E3010008E3010008E301000870
:1000E000E3010008E3010008E3010008E301000860
:1000F000E3010008E3010008E3010008E301000850
:10010000E3010008E301000819390008E3010008D1
:10011000E301000805390008E3010008E3010008D5
:10012000E3010008E3010008E3010008E30100081F
:10013000E3010008E3010008E3010008E30100080F
:10014000E3010008E3010008E3010008FD2D0008B9
:10015000E3010008E3010008E3010008E3010008EF
:10016000E3010008E3010008E3010008E3010008DF
:10017000E3010008E3010008E3010008E3010008CF
:10018000E3010008E3010008E3010008E3010008BF
:10019000E3010008E3010008E3010008E3010008AF
:1001A000E3010008E3010008E3010008E30100089F
:1001B000E3010008E3010008E3010008E30100088F
:1001C000E3010008E3010008E3010008E30100087F
:1001D000E3010008E3010008E3010008E30100086F
:1001E00002E000F000F8FEE772B6374880F30888B6
:1001F000364880F3098836483649086040F20000E6
:10020000CCF200004EF63471CEF200010860BFF36C
:100210004F8FBFF36F8F40F20000C0F2F0004EF638
:100220008851CEF200010860BFF34F8FBFF36F8F8C
:100230004FF00000E1EE100A4EF63C71CEF20001E4
:100240000860062080F31488BFF36F8F02F09EFAD7
:1002500003F09EF94FF055301F491B4A91423CBFB5
:1002600041F8040BFAE71D49184A91423CBF41F896
:10027000040BFAE71A491B4A1B4B9A423EBF51F83E
:10028000040B42F8040BF8E700201849184A914281
:100290003CBF41F8040BFAE702F07CFA03F0CCF91A
:1002A000144C154DAC4203DA54F8041B8847F9E7A7
:1002B00000F042F8114C124DAC4203DA54F8041B22
:1002C0008847F9E702F064BA000600200022002007
:1002D0000000000808ED00E00000002000060020FB
:1002E000283D0008002200204C220020502200203F
:1002F000A0300020E0010008E0010008E001000853
:10030000E00100082DE9F04F2DED108AC1F80CD066
:10031000C3689D46BDEC108ABDE8F08F002383F3CF
:1003200011882846A047002001F0BEFDFEE701F03D
:1003300047FD00DFFEE7000038B500F0E3FB02F008
:10034000F5F940B1164B6FF03F01002259720F21B1
:100350001A729972DA7202F0CFF9054602F008FAC1
:100360000446C8B90F4B9D4218D001339D4218BFB7
:10037000044641F2883504BF01240025002002F024
:10038000C5F90CB100F074F800F02EFD284600F01D
:10039000BFF800F06DF8F9E70025EFE70546EDE757
:1003A00000220020010007B008B500F077FBA0F1A3
:1003B00020035842584108BD07B5042101900DEBB8
:1003C000010000F089FB03B05DF804FB38B5302371
:1003D00083F31188174803680BB101F031FE164A08
:1003E000144800234FF47A7101F020FE002383F3B8
:1003F0001188124C236813B12368013B23606368A2
:1004000013B16368013B63600D4D2B7833B96368AA
:100410007BB9022000F04AFC322363602B78032B67
:1004200007D163682BB9022000F040FC4FF47A73C7
:10043000636038BD50220020CD03000870230020E7
:1004400068220020084B187003280CD8DFE800F061
:1004500008050208022000F019BC022000F008BCC8
:10046000024B00225A60704768220020702300204F
:10047000234B244A10B51C46196801313FD0043380
:100480009342F9D16268A24239D31F4B9B6803F1B2
:10049000006303F580439A4231D2002000F04CFB08
:1004A0000220FFF7CFFF194B1A6C00221A64196E55
:1004B0001A66196E596C5A64596E5A665A6E5A69A0
:1004C00042F080025A615A6922F080025A615A69E8
:1004D0001A6942F000521A611A6922F000521A6138
:1004E0001B6972B64FF0E0233021C3F8084DD4E900
:1004F000003281F311889D4683F30888104710BDB0
:10050000004000082040000800220020003802407F
:100510002DE9F04F95B0DFF8049302902022FF21DF
:1005200004A8D9F8085000F009FCB34A1378A3B91D
:10053000B248012103601170302383F311880368EE
:100540000BB101F07DFDAE4AAC4800234FF47A7147
:1005500001F06CFD002383F31188029B13B1A94BBA
:10056000029A1A60A84A029C1378032B1EBF00232C
:100570001370A44A4FF0000B18BF5360CDF804B0BD
:100580005E46DA46012000F081FB24B19D4B1B68DA
:10059000002B00F01082002000F080FA071EF4DB30
:1005A000012000F065FBA7F121001628EAD801A37D
:1005B00053F820F0110600082D060008BB060008BD
:1005C0008505000885050008850500083F07000827
:1005D0002D090008210800087D080008A30800086C
:1005E000C908000885050008DB080008FF080008A6
:1005F000750900089906000885050008BD0900086E
:100600001D06000899060008850500087D080008F9
:100610000220FFF7C9FE002840F0FA81029B7B48C8
:10062000BBF1000F08BF1C46022140E04FF47A7076
:1006300000F034FA071EF1DB0220FFF7B5FE0028B8
:10064000ECD0013F052F00F2E581DFE807F003075A
:100650000A0D10330520FFF7AFFE14E0D9F80000B3
:10066000F9E7D9F80400F6E7D9F80800F3E74FF006
:100670001C08404600F062FA08F10408FFF79CFEEF
:10068000B8F12C0FF5D1019B012000FA07F71F43A9
:10069000FBB201934FF0000A00F09CFB2EB1019BCE
:1006A00003F00B030B2B08BF00245948022100F074
:1006B00013FA67E7D9F80C00CDE7002EAED0019B06
:1006C00003F00B030B2BA9D10220FFF76DFE0746A9
:1006D0000028A3D0012000F02FFA0220FFF7B2FE7D
:1006E00000261FFA86F8404600F036FA044670B13C
:1006F0000021404600F040FA01360028F1D1BB4607
:1007000004464448022100F0E7F93E463AE701205A
:10071000FFF798FE2546D9F80830AB4207D928469E
:1007200000F00CFA013040F078810435F3E7364BE5
:1007300000251D70334BBB465D603E46ACE7002E86
:100740003FF46CAF019B03F00B030B2B7FF466AF00
:100750000220FFF777FE322000F0A0F9B0F1000888
:10076000FFF65CAF18F003077FF458AFD9F8082004
:1007700008EB050393423FF651AFB8F5807F3FF792
:100780004DAF254B0393B8450BDD4FF47A7000F065
:1007900085F90028FFF642AF039B013703F8010BF0
:1007A000F0E7C820FFF700FE074600283FF436AF09
:1007B0001F2D11D8C5F12002424504AB25F00300DE
:1007C00028BF424614490392184400F091FA039A54
:1007D0001148FF2100F0B2FA4FEAA8030E49039333
:1007E000C8F38702284600F0B1FA0646002888D0F0
:1007F000039B05EB83054FE76C230020502200206C
:10080000CD030008702300206822002094390008DE
:100810008C390008903900086C220020002200204A
:100820000220FFF7C1FD00283FF4F8AE00F0D0F938
:1008300000283FF4F3AE0027B846D9F80830BB4291
:1008400018D91F2F11D8049B01330ED027F00303B2
:1008500014AA134453F8403C0C93404604220CA9BC
:1008600000F01EFB04378046E7E7384600F066F9E3
:100870000C90F2E74046FFF79FFD0DE7002364214F
:100880000CA80C9300F01EF900287FF4C7AE0220DC
:10089000FFF78AFD00283FF4C1AE0C9800F080F904
:1008A000E9E7002364210CA80C9300F00BF9002861
:1008B0007FF4B4AE0220FFF777FD00283FF4AEAE20
:1008C0000C9800F07DF9D6E70220FFF76DFD0028B7
:1008D0003FF4A4AE00F08CF9CDE70220FFF764FDF1
:1008E00000283FF49BAE0CA9142000F087F9039078
:1008F000FFF762FD03990CA800F0EEF8CCE60220A9
:10090000FFF752FD00283FF489AE464B0CAF03F1D0
:10091000100C186859683A4603C2083363451746F5
:10092000F7D11020FFF748FD1021E4E7322000F056
:10093000B5F8071EFFF672AEBB077FF46FAED9F8AD
:10094000082007EB0A0393423FF668AE0220FFF748
:100950002BFD00283FF462AE27F003075744BA4549
:100960003FF49AAE504600F0E9F8FFF725FD0AF192
:10097000040AF4E74FF47A70FFF716FD00283FF4FD
:100980004DAE00F025F9002849D0049B01330BD06F
:10099000082204A9002000F0D9F900283FD0202225
:1009A000FF2104A800F0CAF91F48022100F094F8C2
:1009B0001E4801F07FFA15B0BDE8F08F002E3FF41D
:1009C0002DAE019B03F00B030B2B7FF427AE00230E
:1009D00064210CA80C9300F075F8074600287FF4FA
:1009E0001DAE0220FFF7E0FC804600283FF416AE63
:1009F00002210D4800F070F841F2883001F05AFAF7
:100A00000C9800F02BFA464600F0E4F93C46B9E5B4
:100A1000064641E64FF0000A00E6BB4671E637465F
:100A20006FE600BF783900088C390008A086010005
:100A30002DE9F84F4FF47A73DFF85880DFF85890BB
:100A400006460D4602FB03F7002498F900305A1CB5
:100A50005FFA84FA01D0A34212D159F82400036846
:100A60002A46D3F820B031463B46D847854207D1C5
:100A7000074B012083F800A0BDE8F88F0124E4E7CC
:100A8000002CFBD04FF4FA7001F014FA0020F3E7C9
:100A9000B8230020102200201422002007B50023D4
:100AA000024601210DF107008DF80730FFF7C0FF66
:100AB00020B19DF8070003B05DF804FB4FF0FF3054
:100AC000F9E700000A4608B50421FFF7B1FF80F0FE
:100AD0000100C0B2404208BD30B4074B0A46197845
:100AE000064B53F821402368DD69054B0146AC46AF
:100AF000204630BC604700BFB823002014220020ED
:100B0000A086010070B501F0F5FC094E094D30805A
:100B1000002428683388834208D901F0E5FC2B685B
:100B200004440133B4F5804F2B60F2D370BD00BF95
:100B3000BA2300207823002001F092BD00F100606C
:100B400000F580400068704700F10060920000F5F9
:100B5000804001F01DBD0000054B1A68054B1B8845
:100B60009B1A834202D9104401F0BEBC002070479A
:100B700078230020BA23002038B5084D044629B157
:100B800028682044BDE8384001F0CEBC28682044E5
:100B900001F0B2FC0028F3D038BD00BF782300205C
:100BA00010F003030AD1B0F5047F05D200F1005024
:100BB000A0F51040D0F80038184670470023FBE736
:100BC00000F10050A0F51040D0F8100A7047000066
:100BD000064991F8243033B10023086A81F82430A3
:100BE0000822FFF7B1BF0120704700BF7C2300201F
:100BF000014B1868704700BF002004E070B5194B26
:100C00001D68194B0138C5F30B0408442D0C042250
:100C10001E88A6420BD15C680A46013C82421346FC
:100C20000FD214F9016F4EB102F8016BF6E7013AE9
:100C300003F10803ECD181420B4602D22C2203F8C7
:100C4000012B0A4A05241688AE4204D1984284BF7B
:100C5000967803F8016B013C02F10402F3D1581AB3
:100C600070BD00BF002004E0D8390008C439000876
:100C7000022803D1044B08229A6170470128FCD155
:100C8000014B0422F8E700BF00100240022804D103
:100C9000054B4FF400229A6170470128FCD1024BAA
:100CA0004FF48022F7E700BF00100240022805D170
:100CB000064A536983F00803536170470128FCD149
:100CC000024A536983F00403F6E700BF00100240B4
:100CD00070B504464FF47A764CB1412C254628BFB6
:100CE000412506FB05F001F0E5F8641BF4E770BD53
:100CF00010B50023934203D0CC5CC4540133F9E710
:100D000010BD000010B5013810F9013F3BB191F959
:100D100000409C4203D11AB10131013AF4E71AB103
:100D200091F90020981A10BD1046FCE703460246D0
:100D3000D01A12F9011B0029FAD170470244034668
:100D4000934202D003F8011BFAE770472DE9F843FC
:100D50001F4D144695F824200746884652BBDFF8FD
:100D600070909CB395F824302BB92022FF2148467F
:100D70002F62FFF7E3FF95F82400C0F10802A242BA
:100D800028BF2246D6B24146920005EB8000FFF70D
:100D9000AFFF95F82430A41B1E44F6B2082E17446A
:100DA0009044E4B285F82460DBD1FFF711FF0028FE
:100DB000D7D108E02B6A03EB82038342CFD0FFF741
:100DC00007FF0028CBD10020BDE8F8830120FBE716
:100DD0007C230020024B1A78024B1A70704700BF28
:100DE000B82300201022002038B5174C174D20469C
:100DF00000F0B6FB2946204600F0DEFB2D686A6D48
:100E0000936B23F4002393634FF47A70FFF760FF32
:100E10000F49284600F0D6FC6A6D0E4D936B28688A
:100E20000D4943F400239363A0424FF4E1330B6078
:100E300001D000F0F5FA6868A04204D0BDE838405F
:100E4000054900F0EDBA38BD98280020E03A0008C6
:100E5000E83A000814220020A423002070B50C4BAF
:100E60000C4D1E780C4B55F826209A4204460DD0A6
:100E70000A4B002114221846FFF760FF0460014668
:100E800055F82600BDE8704000F0CABA70BD00BF3A
:100E9000B82300201422002098280020A42300203A
:100EA00030B5094D0A4491420DD011F8013B58402C
:100EB000082340F30004013B2C4013F0FF0384EAB5
:100EC0005000F6D1EFE730BD2083B8ED02684368EB
:100ED0001143016003B1184770470000024AD3680C
:100EE00043F0C003D36070470050004010B5054C7C
:100EF000054A0021204600F071FA044A044BC4E977
:100F0000972310BDBC230020DD0E000800500040D8
:100F100080DE8002234A037C002918BF0A46012B89
:100F200030B5C0F868220CD11F4B984209D11F4B35
:100F3000196C41F480111964196E41F4801119661D
:100F40001B6EB2F904501468D0F86032D0F85C120D
:100F5000002D03EB5403B3FBF4F3BEBF23F00705EE
:100F600003F0070343EA450394888B60D38843F07A
:100F700040030B61138943F001034B6144F40453B4
:100F800043F02C03CB6004F4A05400230B60B4F5B1
:100F9000806F0B684B680CBF7F23FF2380F864329F
:100FA00030BD00BFF8390008BC23002000380240E3
:100FB0002DE9F041D0F85C62F7683368DA05044641
:100FC0009DB20DD5302383F311884FF48061043036
:100FD000FFF77CFF6FF480733360002383F3118885
:100FE000302383F3118804F1040815F02F033AD15C
:100FF00083F31188380615D5290613D5302383F3DA
:10100000118804F1380000F065F900284EDA082153
:10101000201DFFF75BFF4FF67F733B40F36000231B
:1010200083F311887A0616D56B0614D5302383F323
:101030001188D4E913239A420AD1236C43B127F0D3
:1010400040073F041021201D3F0CFFF73FFFF760D2
:10105000002383F31188D4F86822D36843B3BDE832
:10106000F041106918472B0714D015F0080F0CBF7A
:1010700000214FF48071E80748BF41F02001AA0722
:1010800048BF41F040016B0748BF41F08001404636
:10109000FFF71CFFAD06736805D594F8641220466F
:1010A000194000F0CBF93568ADB29EE77060B6E745
:1010B000BDE8F081F8B5154682680669AA420B467C
:1010C000816938BF8568761AB54204460BD2184646
:1010D0002A46FFF70DFEA3692B44A361A3685B1B9F
:1010E000A3602846F8BD0CD918463246FFF700FE2B
:1010F000AF1BE1683A463044FFF7FAFDE3683B4432
:10110000EBE718462A46FFF7F3FDE368E5E7000042
:1011100083689342F7B51546044638BF8568D0E921
:101120000460361AB5420BD22A46FFF7E1FD636927
:101130002B446361A36828465B1BA36003B0F0BD2A
:101140000DD932460191FFF7D3FD0199E068AF1B3D
:101150003A463144FFF7CCFDE3683B44E9E72A46D1
:10116000FFF7C6FDE368E4E710B50A440024C36155
:10117000029B8460C0E90000C0E90511C160026102
:10118000036210BD08B5D0E90532934201D18268EF
:1011900082B98268013282605A1C42611970D0E9BA
:1011A00004329A4224BFC3684361002100F09EFECE
:1011B000002008BD4FF0FF30FBE7000070B5302382
:1011C00004460E4683F31188A568A5B1A368A269F9
:1011D000013BA360531CA36115782269934224BF8D
:1011E000E368A361E3690BB120469847002383F3CA
:1011F0001188284607E03146204600F067FE0028A7
:10120000E2DA85F3118870BD2DE9F74F04460E46EA
:1012100017469846D0F81C904FF0300A8AF3118890
:101220004FF0000B154665B12A4631462046FFF7C0
:1012300041FF034660B94146204600F047FE0028C2
:10124000F1D0002383F31188781B03B0BDE8F08F41
:10125000B9F1000F03D001902046C847019B8BF3E2
:101260001188ED1A1E448AF31188DCE7C0E90511E4
:10127000C160C3611144009B8260C0E9000001614C
:1012800003627047F8B504460D461646302383F3D3
:101290001188A768A7B1A368013BA36063695A1CC2
:1012A00062611D70D4E904329A4224BFE36863612D
:1012B000E3690BB120469847002080F3118807E0CE
:1012C0003146204600F002FE0028E2DA87F311885A
:1012D000F8BD0000D0E905239A4210B501D182681B
:1012E0007AB98268013282605A1C82611C78036973
:1012F0009A4224BFC3688361002100F0F7FD2046B5
:1013000010BD4FF0FF30FBE72DE9F74F04460E46C6
:1013100017469846D0F81C904FF0300A8AF311888F
:101320004FF0000B154665B12A4631462046FFF7BF
:10133000EFFE034660B94146204600F0C7FD002895
:10134000F1D0002383F31188781B03B0BDE8F08F40
:10135000B9F1000F03D001902046C847019B8BF3E1
:101360001188ED1A1E448AF31188DCE7026843688D
:101370001143016003B11847704700001430FFF7B4
:1013800043BF00004FF0FF331430FFF73DBF0000B4
:101390003830FFF7B9BF00004FF0FF333830FFF7A8
:1013A000B3BF00001430FFF709BF00004FF0FF315A
:1013B0001430FFF703BF00003830FFF763BF0000B1
:1013C0004FF0FF323830FFF75DBF0000012914BF36
:1013D0006FF0130000207047FFF788BD37B5154642
:1013E0000E4A026000224260C0E902220122044645
:1013F00002740B46009000F15C014FF480721430CF
:10140000FFF7B2FE00942B464FF4807204F5AE71E4
:1014100004F13800FFF72AFF03B030BD0C3A000892
:1014200010B53023044683F31188FFF773FD0223C0
:101430002374002080F3118810BD000038B5C36903
:1014400004460D461BB904210844FFF78FFF2946C7
:1014500004F11400FFF796FE002806DA201D4FF471
:101460000061BDE83840FFF781BF38BD02684368BE
:101470001143016003B118477047000013B5446B76
:10148000D4F894341A681178042915D1217C0229E2
:1014900012D11979128901238B4013420CD101A971
:1014A00004F14C0001F02AFFD4F89444019B217907
:1014B0000246206800F0D0F902B010BD143001F0EF
:1014C000ADBE00004FF0FF33143001F0A7BE0000A6
:1014D0004C3001F07FBF00004FF0FF334C3001F083
:1014E00079BF0000143001F07BBE00004FF0FF31E7
:1014F000143001F075BE00004C3001F04BBF00000D
:101500004FF0FF324C3001F045BF00000020704723
:1015100010B5D0F894341A6811780429044617D10C
:10152000017C022914D15979528901238B4013423D
:101530000ED1143001F00EFE024648B1D4F89444A6
:101540004FF4807361792068BDE8104000F072B9F3
:1015500010BD0000406BFFF7DBBF000070470000CC
:101560007FB5124B036000234360C0E902330125BD
:1015700002260F4B057404460290019300F1840289
:10158000294600964FF48073143001F0BFFD094BDB
:101590000294CDE9006304F523724FF48073294669
:1015A00004F14C0001F086FE04B070BD343A00082E
:1015B000551500087D1400080B68302282F311884D
:1015C0000A7903EB820290614A79093243F82200DA
:1015D0008A7912B103EB820398610223C0F8941454
:1015E0000374002080F311887047000038B5037F32
:1015F000044613B190F85430ABB9201D01250221E7
:10160000FFF734FF04F1140025776FF0010100F0BB
:1016100079FC84F8545004F14C006FF00101BDE8EE
:10162000384000F06FBC38BD10B5012104460430CD
:10163000FFF71CFF0023237784F8543010BD00000F
:1016400038B504460025143001F078FD04F14C0053
:10165000257701F047FE201D84F854500121FFF743
:1016600005FF2046BDE83840FFF752BF90F84430F0
:1016700003F06003202B07D190F84520212A4FF07A
:10168000000303D81F2A06D800207047222AFBD166
:10169000C0E90E3303E0034A82630722C263036496
:1016A000012070471C22002037B5D0F894341A6806
:1016B0001178042904461AD1017C022917D119791D
:1016C000128901238B40134211D100F14C052846A9
:1016D00001F0C8FE58B101A9284601F00FFED4F868
:1016E0009444019B21790246206800F0B5F803B0CC
:1016F00030BD0000F0B500EB810385B09E69044663
:101700000D46FEB1302383F3118804EB8507301DAD
:101710000821FFF7ABFEFB685B691B6806F14C0014
:101720001BB1019001F0F8FD019803A901F0E6FD5D
:10173000024648B1039B2946204600F08DF800235D
:1017400083F3118805B0F0BDFB685A691268002A5E
:10175000F5D01B8A013B1340F1D104F14402EAE7C2
:10176000093138B550F82140DCB1302383F31188BA
:10177000D4F894241368527903EB8203DB689B69E5
:101780005D6845B104216018FFF770FE294604F139
:10179000140001F0E9FC2046FFF7BAFE002383F3B2
:1017A000118838BD7047000001F048B8012303706C
:1017B0000023C0E90133C36183620362C3624362F1
:1017C0000363704738B50446302383F3118800253E
:1017D000C0E90355C0E90555416001F03FF8022317
:1017E000237085F31188284638BD000070B500EBE2
:1017F000810305465069DA600E46144618B110227E
:101800000021FFF79BFAA06918B110220021FFF711
:1018100095FA31462846BDE8704001F0E9B800006D
:10182000826802F0011282600022C0E90422826113
:1018300001F06AB9F0B400EB81044789E46801253E
:10184000A4698D403D43458123600023A26063600D
:10185000F0BC01F085B90000F0B400EB8104078909
:10186000E468012564698D403D43058123600023C0
:10187000A2606360F0BC01F0FFB9000070B5022304
:10188000002504460370C0E90255C0E90455C5644B
:10189000856180F8345001F047F863681B6823B114
:1018A00029462046BDE87040184770BD0378052BD7
:1018B00010B504460AD080F8503005230370436801
:1018C0001B680BB1042198470023A36010BD0000E2
:1018D0000178052906D190F85020436802701B68F2
:1018E00003B118477047000070B590F834300446D3
:1018F00013B1002380F8343004F14402204601F093
:1019000025F963689B68B3B994F8443013F0600517
:1019100035D00021204601F0C5FB0021204601F012
:10192000B7FB63681B6813B106212046984706235E
:1019300084F8343070BD204698470028E4D0B4F8CD
:101940004A30E26B9A4288BFE36394F94430E56B16
:10195000002B4FF0300380F20381002D00F0F28065
:10196000092284F8342083F311880021D4E90E235E
:101970002046FFF771FF002383F31188DAE794F81C
:10198000452003F07F0343EA022340F202329342F0
:1019900000F0C58021D8B3F5807F48D00DD8012B49
:1019A0003FD0022B00F09380002BB2D104F14C0207
:1019B000A2630222E2632364C1E7B3F5817F00F0F2
:1019C0009B80B3F5407FA4D194F84630012BA0D181
:1019D000B4F84C3043F0020332E0B3F5006F4DD061
:1019E00017D8B3F5A06F31D0A3F5C063012B90D801
:1019F000636894F846205E6894F84710B4F848305D
:101A00002046B047002884D04368A3630368E3639B
:101A10001AE0B3F5106F36D040F6024293427FF4DD
:101A200078AF5C4BA3630223E3630023C3E794F81E
:101A30004630012B7FF46DAFB4F84C3023F0020335
:101A4000C4E90E55A4F84C30256478E7B4F8443066
:101A5000B3F5A06F0ED194F8463084F84E3020468E
:101A600000F0BAFF63681B6813B101212046984754
:101A7000032323700023C4E90E339CE704F14F03D2
:101A8000A3630123C3E72378042B10D1302383F30E
:101A900011882046FFF7C4FE85F31188032163688F
:101AA00084F84F5021701B680BB12046984794F87A
:101AB0004630002BDED084F84F3004232370636857
:101AC0001B68002BD6D0022120469847D2E794F815
:101AD00048301D0603F00F0120460AD501F028F812
:101AE000012804D002287FF414AF2B4B9AE72B4B2C
:101AF00098E701F00FF8F3E794F84630002B7FF4F5
:101B000008AF94F8483013F00F01B3D01A062046FE
:101B100002D501F0DBFAADE701F0CEFAAAE794F8BE
:101B20004630002B7FF4F5AE94F8483013F00F01E7
:101B3000A0D01B06204602D501F0B4FA9AE701F0C6
:101B4000A7FA97E7142284F8342083F311882B46F0
:101B50002A4629462046FFF76DFE85F31188E9E6FF
:101B60005DB1152284F8342083F311880021D4E973
:101B70000E232046FFF75EFEFDE60B2284F834209C
:101B800083F311882B462A4629462046FFF764FE38
:101B9000E3E700BF643A00085C3A0008603A0008D6
:101BA00038B590F834300446002B3ED0063BDAB20C
:101BB0000F2A34D80F2B32D8DFE803F03731310841
:101BC000223231313131313131313737C56BB0F8F3
:101BD0004A309D4214D2C3681B8AB5FBF3F203FB63
:101BE00012556DB9302383F311882B462A462946B6
:101BF000FFF732FE85F311880A2384F834300EE0B3
:101C0000142384F83430302383F3118800231A46D8
:101C100019462046FFF70EFE002383F3118838BDD6
:101C2000036C03B198470023E7E70021204601F049
:101C300039FA0021204601F02BFA63681B6813B1C2
:101C40000621204698470623D7E7000010B590F8F4
:101C50003430142B044629D017D8062B05D001D8D0
:101C60001BB110BD093B022BFBD80021204601F01F
:101C700019FA0021204601F00BFA63681B6813B1C2
:101C8000062120469847062319E0152BE9D10B239E
:101C900080F83430302383F3118800231A46194624
:101CA000FFF7DAFD002383F31188DAE7C3689B6945
:101CB0005B68002BD5D1036C03B19847002384F8EF
:101CC0003430CEE700230375826803691B68996886
:101CD0009142FBD25A6803604260106058607047BE
:101CE00000230375826803691B6899689142FBD8D9
:101CF0005A680360426010605860704708B5084633
:101D0000302383F311880B7D032B05D0042B0DD0DA
:101D10002BB983F3118808BD8B6900221A604FF03C
:101D2000FF338361FFF7CEFF0023F2E7D1E90032F2
:101D300013605A60F3E70000FFF7C4BF38B50A4BE1
:101D4000DD681C68287522681A605360DC60A3682F
:101D500001229342227501D100F014FD294620464C
:101D6000BDE83840FEF7CEBA2826002030B50C4B2F
:101D7000DD684B1C87B004460FD02B46094A6846E5
:101D800000F054F92046FFF7D9FF009B13B16846D5
:101D900000F056F9A86907B030BDFFF7CFFFF9E7AB
:101DA00028260020FD1C0008044B1A68DB68906898
:101DB0009B68984294BF002001207047282600208D
:101DC00038B50B4B1C68DD6822681A60536001222D
:101DD0002275DC60AB68934201D100F0D5FC284647
:101DE000FFF77EFF01462046BDE83840FEF78ABA7D
:101DF0002826002038B5074C07490848012300254C
:101E00002370656001F06CFB0223237085F3118859
:101E100038BD00BF902800206C3A0008282600201A
:101E200000F044B9034A516853685B1A9842FBD8E2
:101E3000704700BF001000E08B60022308618B82B6
:101E4000084670478368A3F1840243F8142C0269A2
:101E500043F8442C426943F8402C094A43F8242CA7
:101E6000C26843F8182C022203F80C2C002203F855
:101E70000B2C044A43F8102CA3F12000704700BF3C
:101E80001D0300082826002008B5FFF7DBFFBDE88A
:101E90000840FFF751BF0000024BDB6898610F203C
:101EA000FFF74CBF28260020302383F31188FFF76B
:101EB000F3BF000008B50146302383F311880820E2
:101EC000FFF754FF002383F3118808BD064BDB683E
:101ED00039B1426818605A60136043600420FFF70C
:101EE00045BF4FF0FF307047282600200368984216
:101EF00006D01A680260506099611846FFF71CBF4F
:101F00007047000038B504460D462068844200D171
:101F100038BD036823605C608561FFF70DFFF4E75F
:101F200010B503689C68A2420CD85C688A600B609C
:101F30004C602160596099688A1A9A604FF0FF33AB
:101F4000836010BD1B68121BECE700000A2938BF34
:101F50000A2170B504460D460A26601901F0B8FA48
:101F600001F0A0FA041BA54203D8751C2E460446B6
:101F7000F3E70A2E04D9BDE87040012001F0F0BA61
:101F800070BD0000F8B5144B0D46D96103F1100186
:101F900041600A2A1969826038BF0A2201604860DC
:101FA0001861A818144601F083FA0A2701F07AFA9A
:101FB000431BA342064606D37C1C281901F088FA6D
:101FC00027463546F2E70A2F04D9BDE8F84001203C
:101FD00001F0C6BAF8BD00BF28260020F8B50646B5
:101FE0000D4601F05FFA0F4A134653F8107F9F42E7
:101FF00006D12A4601463046BDE8F840FFF7C2BF89
:10200000D169BB68441A2C1928BF2C46A34202D9B7
:102010002946FFF79BFF224631460348BDE8F840BA
:10202000FFF77EBF282600203826002010B4C0E924
:10203000032300235DF8044B4361FFF7CFBF00008B
:1020400010B5194C236998420DD0D0E9003281684F
:1020500013605A609A680A449A60002303604FF044
:10206000FF33A36110BD2346026843F8102F53606D
:102070000022026022699A4203D1BDE8104001F0BB
:1020800021BA936881680B44936001F00BFA2269CE
:10209000E1699268441AA242E4D91144BDE81040B3
:1020A000091AFFF753BF00BF282600202DE9F0478B
:1020B000DFF8BC8008F110072C4ED8F8105001F062
:1020C000F1F9D8F81C40AA68031B9A423ED8144480
:1020D000D5E900324FF00009C8F81C4013605A607F
:1020E000C5F80090D8F81030B34201D101F0EAF9F8
:1020F00089F31188D5E9033128469847302383F3C3
:1021000011886B69002BD8D001F0CCF96A69A0EB7B
:1021100004094A4582460DD2022001F021FA00222C
:10212000D8F81030B34208D151462846BDE8F047F0
:10213000FFF728BF121A2244F2E712EB090938BF51
:102140004A4629463846FFF7EBFEB5E7D8F8103087
:10215000B34208D01444211AC8F81C00A960BDE895
:10216000F047FFF7F3BEBDE8F08700BF3826002038
:102170002826002000207047FEE70000704700007E
:102180004FF0FF307047000002290CD0032904D023
:102190000129074818BF00207047032A05D80548C1
:1021A00000EBC2007047044870470020704700BF32
:1021B000443B00082C220020F83A000870B59AB081
:1021C0000546084601A9144600F0C2F801A8FEF72A
:1021D000ADFD431C5B00C5E90034002223700323DE
:1021E0006370C6B201AB02341046D1B28E4204F124
:1021F000020401D81AB070BD13F8011B04F8021CC8
:1022000004F8010C0132F0E708B5302383F311889C
:102210000348FFF749FA002383F3118808BD00BF84
:102220009828002090F8443003F01F02012A07D1BB
:1022300090F845200B2A03D10023C0E90E3315E0A6
:1022400003F06003202B08D1B0F848302BB990F888
:102250004520212A03D81F2A04D8FFF707BA222ACB
:10226000EBD0FAE7034A82630722C26303640120CA
:10227000704700BF2322002007B5052917D8DFE8E3
:1022800001F0191603191920302383F31188104A1D
:1022900001900121FFF7AAFA01980E4A0221FFF7E7
:1022A000A5FA0D48FFF7CCF9002383F3118803B09A
:1022B0005DF804FB302383F311880748FFF796F994
:1022C000F2E7302383F311880348FFF7ADF9EBE71A
:1022D000983A0008BC3A00089828002038B50C4D00
:1022E0000C4C0D492A4604F10800FFF767FF05F181
:1022F000CA0204F110000949FFF760FF05F5CA7230
:1023000004F118000649BDE83840FFF757BF00BF89
:10231000602D00202C220020783A0008823A000824
:102320008D3A000870B5044608460D46FEF7FEFCDF
:10233000C6B22046013403780BB9184670BD324648
:102340002946FEF7DFFC0028F3D10120F6E7000064
:102350002DE9F04705460C46FEF7E8FC2B49C6B2CE
:102360002846FFF7DFFF08B10736F6B228492846AE
:10237000FFF7D8FF08B11036F6B2632E0BD8DFF89E
:102380008C80DFF88C90234FDFF894A02E7846B92C
:102390002670BDE8F08729462046BDE8F04701F0E9
:1023A000E3BA252E2ED1072241462846FEF7AAFC85
:1023B00070B9194B224603F10C0153F8040B42F893
:1023C000040B8B42F9D11B88138007350E34DDE7EF
:1023D000082249462846FEF795FC98B90F4BA21CE7
:1023E000197809090232C95D02F8041C13F8011BAF
:1023F00001F00F015345C95D02F8031CF0D11834F8
:102400000835C3E704F8016B0135BFE7643B0008FA
:102410008D3A00087B3B00086C3B0008107AFF1FD8
:102420001C7AFF1FBFF34F8F024AD368DB03FCD433
:10243000704700BF003C024008B5094B1B7873B9D8
:10244000FFF7F0FF074B1A69002ABFBF064A5A6020
:1024500002F188325A601A6822F480621A6008BD5C
:10246000BE2F0020003C02402301674508B50B4BFE
:102470001B7893B9FFF7D6FF094B1A6942F0004267
:102480001A611A6842F480521A601A6822F4805263
:102490001A601A6842F480621A6008BDBE2F0020DC
:1024A000003C02401728F0B516D80C4C0C49237894
:1024B0007BB90C4D0E4618234FF0006255F8047B93
:1024C00046F8042B013B13F0FF033A44F6D10123F5
:1024D000237051F82000F0BD0020FCE720300020E0
:1024E000C02F00208C3B0008014B53F820007047A0
:1024F0008C3B000818207047172810B5044601D9F6
:10250000002010BDFFF7CEFF064B53F824301844CF
:10251000C21A0BB90120F4E712680132F0D1043B72
:10252000F6E700BF8C3B0008172838B5044628D8CA
:102530001549FFF777FFFFF77FFFF323CB600C23ED
:10254000B0FBF3F203FB1205D30143EAC503DBB290
:1025500043F4007343F002030B610B6943F48033CF
:102560000B61FFF75FFFFFF79DFF084B53F8241047
:1025700000F0DAF8FFF77AFF2046BDE83840FFF7B1
:10258000BBBF002038BD00BF003C02408C3B0008B0
:10259000F8B512F00103144642D18218B2F1026F6D
:1025A00057D82D4B1B6813F0010352D02B4DFFF76A
:1025B00043FFF323EB60FFF735FF40F20127032CC5
:1025C00015D824F001046618244C401A40F2011773
:1025D000B142236900EB010524D123F001032361FB
:1025E000FFF744FF0120F8BD043C0430E7E7830710
:1025F000E7D12B6923F440732B612B693B432B619B
:1026000051F8046B0660BFF34F8FFFF70BFF0368B1
:102610009E42E9D02B6923F001032B61FFF726FFCF
:102620000020E0E723F44073236123693B432361E7
:102630000B882B80BFF34F8FFFF7F4FE2D8831F806
:10264000023BADB2AB42C3D0236923F00103236147
:10265000E4E71846C7E700BF00380240003C0240EC
:10266000084908B50B7828B11BB9FFF7E5FE01232F
:102670000B7008BD002BFCD0BDE808400870FFF7C8
:10268000F5BE00BFBE2F002010B50244064BD2B2EB
:10269000904200D110BD441C00B253F8200041F814
:1026A000040BE0B2F4E700BF502800400F4B30B5F8
:1026B0001C6F240407D41C6F44F400741C671C6F47
:1026C00044F400441C670A4C236843F4807323607D
:1026D0000244084BD2B2904200D130BD441C00B23B
:1026E00051F8045B43F82050E0B2F4E700380240B0
:1026F000007000405028004007B5012201A90020C9
:10270000FFF7C2FF019803B05DF804FB13B5044660
:10271000FFF7F2FFA04205D0012201A90020019499
:10272000FFF7C4FF02B010BD70470000094B5A8884
:10273000B2F5805F10460BD022F0020341F2010295
:10274000934205D041F20703C31A584258417047DB
:1027500001207047002004E0034B1A681AB9034AAD
:10276000D2F874281A6070472430002000300240EC
:1027700008B5FFF7F1FF024B1868C0F3407008BDC1
:1027800024300020704700007047000070470000B0
:10279000FEE700000A4B0B480B4A90420BD30B4B51
:1027A000DA1C121AC11E22F003028B4238BF00222B
:1027B0000021FEF7C3BA53F8041B40F8041BECE7F2
:1027C000743D0008A0300020A0300020A030002080
:1027D00070B5D0E915439E6800224FF0FF3504EB39
:1027E00042135101D3F800090028BEBFD3F80009F5
:1027F00040F08040C3F80009D3F8000B0028BEBFAA
:10280000D3F8000B40F08040C3F8000B013263188E
:102810009642C3F80859C3F8085BE0D24FF00113A1
:10282000C4F81C3870BD0000890141F0200101612D
:1028300003699B06FCD41220FFF7F4BA10B5054CCF
:102840002046FEF7B3FF4FF0A0436365024BA3653C
:1028500010BD00BF28300020103C000870B5037880
:10286000012B054650D12A4B446D98421BD1294B70
:102870005A6B42F080025A635A6D42F080025A65E8
:102880005A6D5A6942F080025A615A6922F08002F8
:102890005A610E2143205B6900F022FC1E4BE3606D
:1028A0001E4BC4F800380023C4F8003EC023236048
:1028B0006E6D4FF45023A3633369002BFCDA0123C0
:1028C00033610C20FFF7AEFA3369DB07FCD412202A
:1028D000FFF7A8FA3369002BFCDA0026A660284629
:1028E000FFF776FF6B68C4F81068DB68C4F81468FB
:1028F000C4F81C684BB90A4BA3614FF0FF33636106
:10290000A36843F00103A36070BD064BF4E700BF6A
:10291000283000200038024040140040030020020C
:10292000003C30C0083C30C0F8B5446D054600217D
:102930002046FFF779FFA96D00234FF001128F6841
:10294000C4F834384FF00066C4F81C284FF0FF304C
:1029500004EB431201339F42C2F80069C2F8006BD6
:10296000C2F80809C2F8080BF2D20B686A6DEB6571
:10297000636210231361166916F01006FBD1122052
:10298000FFF750FAD4F8003823F4FE63C4F8003897
:10299000A36943F4402343F01003A3610923C4F85F
:1029A0001038C4F814380A4BEB604FF0C043C4F839
:1029B000103B084BC4F8003BC4F81069C4F8003958
:1029C000EB6D03F1100243F48013EA65A362F8BDD6
:1029D000EC3B000840800010426D90F84E10D2F899
:1029E000003823F4FE6343EA0113C2F8003870474D
:1029F0002DE9F84300EB8103456DDA68166806F0AF
:102A00000306731E022B05EB41130C4680460FFA9A
:102A100081F94FEA41104FF00001C3F8101B4FF04D
:102A2000010104F1100398BFB60401FA03F39169A0
:102A30008EBF334E06F1805606F5004600293AD087
:102A4000578A04F15801490137436F50D5F81C18D3
:102A50000B43C5F81C382B180021C3F81019536913
:102A60000127611EA7409BB3138A928B9B08012A02
:102A700088BF5343D8F85C20981842EA034301F119
:102A8000400205EB8202C8F85C00214653602846EC
:102A9000FFF7CAFE08EB8900C3681B8A43EA845328
:102AA000483464011E432E51D5F81C381F43C5F825
:102AB0001C78BDE8F88305EB4917D7F8001B21F413
:102AC0000041C7F8001BD5F81C1821EA0303C0E732
:102AD00004F13F0305EB83030A4A5A602846214666
:102AE000FFF7A2FE05EB4910D0F8003923F40043AC
:102AF000C0F80039D5F81C3823EA0707D7E700BF2C
:102B00000080001000040002826D1268C265FFF7A9
:102B10005FBE00005831436D49015B5813F400401B
:102B200004D013F4001F0CBF0220012070470000E6
:102B30004831436D49015B5813F4004004D013F44D
:102B4000001F0CBF022001207047000000EB810134
:102B5000CB68196A0B6813604B68536070470000BC
:102B600000EB810330B5DD68AA691368D36019B939
:102B7000402B84BF402313606B8A1468426D1C4451
:102B8000013CB4FBF3F46343033323F0030302EB90
:102B9000411043EAC44343F0C043C0F8103B2B68E4
:102BA00003F00303012B09B20ED1D2F8083802EB6F
:102BB000411013F4807FD0F8003B14BF43F08053E2
:102BC00043F00053C0F8003B02EB4112D2F8003B47
:102BD00043F00443C2F8003B30BD00002DE9F04152
:102BE000244D6E6D06EB40130446D3F8087BC3F802
:102BF000087B38070AD5D6F81438190706D505EB2F
:102C000084032146DB6828465B689847FA071FD58E
:102C1000D6F81438DB071BD505EB8403D968CCB98B
:102C20008B69488A5A68B2FBF0F600FB16228AB913
:102C30001868DA6890420DD2121AC3E900243023D2
:102C400083F311880B482146FFF78AFF84F311882C
:102C5000BDE8F081012303FA04F26B8923EA020341
:102C60006B81CB68002BF3D021460248BDE8F041D0
:102C7000184700BF2830002000EB810370B5DD68E5
:102C8000436D6C692668E6604A0156BB1A444FF4EE
:102C90000020C2F810092A6802F00302012A0AB2D1
:102CA0000ED1D3F8080803EB421410F4807FD4F857
:102CB000000914BF40F0805040F00050C4F80009F3
:102CC00003EB4212D2F8000940F00440C2F80009B8
:102CD000D3F83408012202FA01F10143C3F8341891
:102CE00070BD19B9402E84BF4020206020682E8A14
:102CF0008419013CB4FBF6F440EAC44040F00050B3
:102D00001A44C6E72DE9F8433B4D6E6D06EB4013C0
:102D10000446D3F80889C3F8088918F0010F4FEA70
:102D200040171AD0D6F81038DB0716D505EB80030C
:102D3000D9684B691868DA68904230D2121A4FF09D
:102D400000091A60C3F80490302383F311882146E8
:102D50002846FFF791FF89F3118818F0800F1CD0E7
:102D6000D6F834380126A640334216D005EB84034A
:102D70006D6DD3F80CC0DCF814200134E4B2D2F845
:102D800000E005EB04342F445168714515D3D5F8A4
:102D9000343823EA0606C5F83468BDE8F883012311
:102DA00003FA04F22B8923EA02032B818B68002BA0
:102DB000D3D0214628469847CFE7BCF81000AEEBA9
:102DC0000103834228BF0346D7F8180980B2B3EB4A
:102DD000800FE2D89068A0F1040959F8048FC4F874
:102DE0000080A0EB09089844B8F1040FF5D8184406
:102DF0000B4490605360C7E7283000202DE9F74F5F
:102E0000A24C656D6E69AB691E4016F480586E6108
:102E100007D02046FEF732FD03B0BDE8F04F00F0CA
:102E20004DBC002E12DAD5F8003E98489B071EBF15
:102E3000D5F8003E23F00303C5F8003ED5F804386A
:102E400023F00103C5F80438FEF742FD370505D528
:102E50008E48FFF7BDFC8D48FEF728FDB0040CD569
:102E6000D5F8083813F0060FEB6823F470530CBF45
:102E700043F4105343F4A053EB6031071BD5636850
:102E8000DB681BB9AB6923F00803AB612378052B22
:102E90000CD1D5F8003E7D489A071EBFD5F8003EFC
:102EA00023F00303C5F8003EFEF712FD6368DB68FC
:102EB0000BB176489847F30274D4B70227D5D4F8FB
:102EC0005490DFF8C8B100274FF0010A09EB471210
:102ED000D2F8003B03F44023B3F5802F11D1D2F890
:102EE000003B002B0DDA62890AFA07F322EA03039A
:102EF000638104EB8703DB68DB6813B1394658460E
:102F00009847A36D01379B68FFB29F42DED9F00658
:102F100017D5676D3A6AC2F30A1002F00F0302F484
:102F2000F012B2F5802F00F08580B2F5402F08D165
:102F300004EB83030022DB681B6A07F5805790428D
:102F40006AD13003D5F8184813D5E10302D5002023
:102F5000FFF744FEA20302D50120FFF73FFE630303
:102F600002D50220FFF73AFE270302D50320FFF720
:102F700035FE75037FF550AFE00702D50020FFF75F
:102F8000C1FEA10702D50120FFF7BCFE620702D5F2
:102F90000220FFF7B7FE23077FF53EAF0320FFF7C0
:102FA000B1FE39E7636DDFF8E4A0019300274FF02D
:102FB0000109A36D9B685FFA87FB9B453FF67DAFD8
:102FC000019B03EB4B13D3F8001901F44021B1F539
:102FD000802F1FD1D3F8001900291BDAD3F800196C
:102FE00041F09041C3F80019D3F800190029FBDB28
:102FF0005946606DFFF718FC218909FA0BF321EAA5
:103000000303238104EB8B03DB689B6813B15946F0
:10301000504698470137CCE7910708BFD7F80080A2
:10302000072A98BF03F8018B02F1010298BF4FEA0B
:10303000182884E7023304EB830207F580575268AF
:10304000D2F818C0DCF80820DCE9001CA1EB0C0C5D
:10305000002188420AD104EB830463689B699A6863
:1030600002449A605A6802445A606AE711F0030FFA
:1030700008BFD7F800808C4588BF02F8018B01F1AA
:10308000010188BF4FEA1828E3E700BF283000207D
:10309000436D03EB4111D1F8003B43F40013C1F839
:1030A000003B7047436D03EB4111D1F8003943F405
:1030B0000013C1F800397047436D03EB4111D1F89B
:1030C000003B23F40013C1F8003B7047436D03EB52
:1030D0004111D1F8003923F40013C1F800397047C9
:1030E00000F1604303F561430901C9B283F800139D
:1030F000012200F01F039A4043099B0003F1604343
:1031000003F56143C3F880211A60704730B5039C12
:103110000172043304FB0325C0E90653049B0363D7
:103120000021059BC160C0E90000C0E90422C0E99C
:103130000842C0E90A11436330BD0000416A002221
:10314000C0E90411C0E90A22C2606FF00101FEF774
:10315000D9BE0000D0E90432934201D1C2680AB955
:10316000181D70470020704703691960C26801325A
:10317000C260C269134482690361934224BF436AF7
:1031800003610021FEF7B2BE38B504460D46E36880
:103190003BB16269131D1268A3621344E36200200D
:1031A00007E0237A33B929462046FEF78FFE002830
:1031B000EDDA38BD6FF00100FBE70000C368C269BB
:1031C000013BC3604369134482694361934224BF56
:1031D000436A436100238362036B03B1184770475E
:1031E00070B53023044683F31188866A3EB9FFF731
:1031F000CBFF054618B186F31188284670BDA36A37
:10320000E26A13F8015BA362934202D32046FFF700
:10321000D5FF002383F31188EFE700002DE9F84F75
:1032200004460E46174698464FF0300989F3118838
:103230000025AA46D4F828B0BBF1000F09D14146B9
:103240002046FFF7A1FF20B18BF311882846BDE887
:10325000F88FD4E90A12A7EB050B521A934528BF41
:103260009346BBF1400F1BD9334601F1400251F8A0
:10327000040B43F8040B9142F9D1A36A4033403662
:10328000A3624035D4E90A239A4202D32046FFF7CD
:1032900095FF8AF31188BD42D8D289F31188C9E716
:1032A00030465A46FDF724FDA36A5B445E44A362A0
:1032B0005D44E7E710B5029C0172043303FB04216F
:1032C000C0E906130023C0E90A33039B0363049B90
:1032D000C460C0E90000C0E90422C0E908424363B9
:1032E00010BD0000026AC260426AC0E904220022E6
:1032F000C0E90A226FF00101FEF704BED0E9042301
:103300009A4201D1C26822B9184650F8043B0B60BA
:10331000704700231846FAE7C368C2690133C360E7
:103320004369134482694361934224BF436A436102
:103330000021FEF7DBBD000038B504460D46E3680A
:103340003BB123691A1DA262E2691344E3620020C3
:1033500007E0237A33B929462046FEF7B7FD002857
:10336000EDDA38BD6FF00100FBE70000036919607A
:10337000C268013AC260C269134482690361934220
:1033800024BF436A036100238362036B03B11847C0
:103390007047000070B530230D460446114683F394
:1033A0001188866A2EB9FFF7C7FF10B186F311881E
:1033B00070BDA36A1D70A36AE26A01339342A362DF
:1033C00004D3E16920460439FFF7D0FF002080F3E1
:1033D0001188EDE72DE9F84F04460D4690469946D1
:1033E0004FF0300A8AF311880026B346A76A4FB916
:1033F00049462046FFF7A0FF20B187F311883046E9
:10340000BDE8F88FD4E90A073A1AA8EB06079742F5
:1034100028BF1746402F1BD905F1400355F8042B50
:1034200040F8042B9D42F9D1A36A4033A362403691
:10343000D4E90A239A4204D3E16920460439FFF70C
:1034400095FF8BF311884645D9D28AF31188CDE7D1
:1034500029463A46FDF74CFCA36A3B443D44A3622F
:103460003E44E5E7D0E904239A4217D1C3689BB1F3
:10347000836A8BB1043B9B1A0ED01360C368013B77
:10348000C360C3691A44836902619A4224BF436AD4
:103490000361002383620123184670470023FBE782
:1034A00000F036B9014B586A704700BF000C00406D
:1034B000034B002258631A610222DA60704700BF92
:1034C000000C0040014B0022DA607047000C004005
:1034D000014B5863704700BF000C0040FEE700003E
:1034E00070B51B4B01630025044686B058608562A9
:1034F0000E4600F0BFF804F11003C4E904334FF0A6
:10350000FF33C4E90635C4E90044A560E562FFF76E
:10351000C9FF2B460246C4E9082304F134010D4AD1
:10352000256580232046FEF787FC0123E0600A4AD8
:103530000375009272680192B268CDE90223074BCD
:103540006846CDE90435FEF79FFC06B070BD00BFAC
:10355000902800201C3C0008213C0008DD340008B5
:10356000024AD36A1843D062704700BF2826002061
:103570004B6843608B688360CB68C3600B694361B1
:103580004B6903628B6943620B68036070470000FC
:1035900008B5264B26481A6940F2FF110A431A6102
:1035A0001A6922F4FF7222F001021A611A691A6B79
:1035B0000A431A631A6D0A431A651E4A1B6D1146A7
:1035C000FFF7D6FF02F11C0100F58060FFF7D0FF86
:1035D00002F1380100F58060FFF7CAFF02F15401E3
:1035E00000F58060FFF7C4FF02F1700100F5806014
:1035F000FFF7BEFF02F18C0100F58060FFF7B8FF16
:1036000002F1A80100F58060FFF7B2FF02F1C401EA
:1036100000F58060FFF7ACFF02F1E00100F580608B
:10362000FFF7A6FFBDE8084000F0F0B80038024000
:1036300000000240283C000808B500F081F9FEF7C0
:10364000D9FBFFF789F8BDE80840FEF747BE000048
:1036500070470000EFF3098305494A6B22F001022D
:103660004A63683383F30988002383F31188704722
:1036700000EF00E0302080F3118862B60C4B0D4A59
:10368000D96821F4E0610904090C0A43DA60D3F82F
:10369000FC20094942F08072C3F8FC200A6842F01D
:1036A00001020A602022DA7783F82200704700BF07
:1036B00000ED00E00003FA05001000E010B5302333
:1036C00083F311880E4B5B6813F4006314D0F1EEA2
:1036D000103AEFF30984683C4FF08073E361094BC3
:1036E000DB6B236684F30988FEF75EFB10B1064BA3
:1036F000A36110BD054BFBE783F31188F9E700BF19
:1037000000ED00E000EF00E02F03000832030008A6
:103710000E4B1A6C42F008021A641A6E42F008024C
:103720001A660B4A1B6E936843F008039360094BBB
:1037300053229A624FF0FF32DA6200229A615A6392
:10374000DA605A6001225A611A60704700380240FC
:10375000002004E0000C0040094A08B51169D36854
:103760000B40D9B2C9439B07116107D5302383F3BE
:103770001188FEF755FB002383F3118808BD00BFB5
:10378000000C00401F4B1A696FEAC2526FEAD25216
:103790001A611A69C2F308021A614FF0FF301A6900
:1037A0005A69586100215A6959615A691A6A62F066
:1037B00080521A621A6A02F080521A621A6A5A6AAF
:1037C00058625A6A59625A6A1A6C42F080521A64F4
:1037D0001A6E42F080521A661A6E0B4A106840F454
:1037E00080701060186F00F44070B0F5007F1EBF4D
:1037F0004FF4803018671967536823F400735360DF
:1038000000F092B80038024000700040344B4FF096
:1038100080521A64334A4FF4404111601A6842F0F2
:1038200001021A601A689107FCD59A6822F0030217
:103830009A602B4B9A6812F00C02FBD1196801F0C8
:10384000F90119609A601A6842F480321A601A68A5
:103850009203FCD55A6F42F001025A67204B5A6F0F
:103860009007FCD5204A5A601A6842F080721A60AC
:103870001C4A53685904FCD5194B1A689201FCD5AF
:103880001A4A9A600322C3F88C20194B1A68194B04
:103890009A42194B21D1194A1168194A91421CD1F7
:1038A00040F205121A60144A136803F00F03052B47
:1038B000FAD10B4B9A6842F002029A609A6802F0C1
:1038C0000C02082AFAD15A6C42F480425A645A6EA9
:1038D00042F480425A665B6E704740F20572E1E73F
:1038E00000380240007000400854400700948838B7
:1038F000002004E011640020003C024000ED00E0E4
:1039000041C20F4108B50348FDF752FBBDE808402E
:10391000FFF7D4BEBC23002008B5FFF71DFFBDE8AC
:103920000840FFF7CBBE000008B507213220FFF7A3
:10393000D7FBBDE808400C213520FFF7D1BB0000C4
:1039400008B5FFF71FFF00F00DF8FDF745FDFDF787
:103950002BFFFDF703FEFFF77BFEBDE80840FFF7F6
:103960009FBD000070470000034611F8012B03F8CB
:10397000012B002AF9D17047343237393864623864
:1039800062343539626232350000000012100000E6
:10399000121100001213000053544D3332463F3FC2
:1039A0003F0053544D3332463430780053544D3336
:1039B00032463432780053544D333246343436581C
:1039C00058000000012033000010410001105A008F
:1039D000031059000710310000000000983900085A
:1039E00013040000A239000819040000AC390008D3
:1039F00021040000B6390008009600000000000015
:103A000000000000000000000000000000000000B6
:103A10009913000885130008C1130008AD130008AE
:103A2000B9130008A5130008911300087D130008BE
:103A3000CD13000800000000D9140008C5140008C8
:103A400001150008ED140008F9140008E514000839
:103A5000D1140008BD1400080D1500080000000076
:103A6000010000000000000063300000683A000818
:103A700080260020902800204172647550696C6F88
:103A8000740025424F415244252D424C0025534598
:103A90005249414C250000000200000000000000D7
:103AA000F51600086117000840004000302D002086
:103AB000402D002002000000000000000300000074
:103AC00000000000A5170008000000001000000022
:103AD000502D002000000000010000000000000048
:103AE0002830002001010200792200088921000805
:103AF000252200080922000843000000003B0008BE
:103B000009024300020100C0320904000001020260
:103B10000100052400100105240100010424020213
:103B20000524060001070582030800FF09040100BF
:103B3000020A00000007050102400000070581029B
:103B400040000000120000004C3B00081201100170
:103B50000200004009124157000201020301000067
:103B60000403090425424F4152442500466C7969FB
:103B70006E674D6F6F6E46343237003031323334FA
:103B8000353637383941424344454600004000004D
:103B90000040000000400000004000000000010064
:103BA000000002000000020000000200000002000D
:103BB00000000200000002000000020000400000BF
:103BC0000040000000400000004000000000010034
:103BD00000000200000002000000020000000200DD
:103BE00000000200000002000000020000000000CF
:103BF000E9180008A11B00084D1C00084000400007
:103C0000883000208830002001000000983000201B
:103C10008000000040010000030000006D61696E3B
:103C20000069646C650000000001802A000000004B
:103C3000AAAAAAAA00010024FFFF000000000000B9
:103C400000A00A001500000100000000AAAAAAA80E
:103C500015000001FFFF0000000000000000000050
:103C60000000000200000000AAAAAAAA00000001A9
:103C7000FFFF00000000000000000800200000001E
:103C800000000000AAAAAAAA10000000FFFF00007E
:103C9000000800000000000050000040000000008C
:103CA000AAAAAAAA00000040FFFF0000000000002E
:103CB000000000000000000000000000AAAAAAAA5C
:103CC00000000000FFFF00000000000000000000F6
:103CD0000000000000000000AAAAAAAA000000003C
:103CE000FFFF0000000000000000000000000000D6
:103CF000000000000A0000000000000003000000B7
:103D000000000000000000000000000000000000B3
:103D100000000000000000000000000000000000A3
:103D200000000000000000002C0400000000000063
:103D300000C01F0000000000FF00000098280020C5
:103D4000BC23002000960000000008009600000040
:103D50000008000004000000603B000800000000B4
:103D60000000000000000000000000000000000053
:043D7000000000004F
:00000001FF
